:0200000480007A
:10000000971700009387070093001000130100006A
:10001000B701F17F9381F1FF370200809302F0FF77
:1000200073100034F3A00034F31000347321013452
:1000300073110034F3A10134F3110034732202343C
:1000400073120034F3A20234F312003423A0070029
:1000500023A2170023A4270023A6370023A84700C4
:1000600023AA570097120000938242FB93051000C9
:1000700013060000B706F17F9386F6FF370700806E
:100080009307F0FF73100034F3A50534732606348C
:10009000F3A6063473270734F3A707347328003414
:1000A00023A0B20023A2C20023A4D20023A6E20010
:1000B00023A8F20023AA0201171D0000130D8DF7DB
:1000C000B75A3412938A8A677310003473AB0A34B8
:1000D000F32B0B34F31B003473AC0B34F32C0034D0
:1000E00023205D0123226D0123247D0123268D0120
:1000F00023289D0197100000938000F5377F7242FE
:10010000130FFFE673100F3473200F3423A0000089
:1001100023A2E00117110000130181F3B79FFFF73D
:10012000938F8F8173900F347320003473200034C9
:10013000F32F0034232001002322F10117110000C6
:10014000130181F1B753163293838349B75238961E
:100150009382422773100034F3A20234F3A30334D2
:1001600073240434232051002322710023248100AE
:1001700017150000130505E997150000938585EE16
:10018000370610F01306C6F26306B5028326C500D3
:100190002320D600832685002320D6008326450011
:1001A0002320D600832605002320D6001305050151
:1001B0006FF09FFD370510F0130505F223200500B1
:0401C000000000003B
:10100000FFFFFFFFFFFFFFFFFFFFFFFFFFFFFFFFF0
:10101000FFFFFFFFFFFFFFFFFFFFFFFFFFFFFFFFE0
:10102000FFFFFFFFFFFFFFFFFFFFFFFFFFFFFFFFD0
:10103000FFFFFFFFFFFFFFFFFFFFFFFFFFFFFFFFC0
:10104000FFFFFFFFFFFFFFFFFFFFFFFFFFFFFFFFB0
:10105000FFFFFFFFFFFFFFFFFFFFFFFFFFFFFFFFA0
:040000058000000077
:00000001FF
